:100000000C946C040C9432330C94B3040C94B3042D
:100010000C94B3040C94B3040C94B3040C94B30484
:100020000C94B3040C94B3040C941B2B0C94D72A9B
:100030000C946E2C0C94B3040C94B3040C94B30481
:100040000C94B3040C94B3040C94B3040C94B30454
:100050000C94B3040C944A2C0C94B3040C94B30485
:100060000C94B3040C94B3040C94B3040C94B30434
:100070000C94B3040C94B3040C94B3040C94B30424
:100080000C94B3040C94B3040C94B3040C94B30414
:100090000C94B3040C94B3040C94B3040C94B30404
:1000A0000C94B3040C94B3040C94B3040631FF090C
:1000B00074A1010975150026FF00952075088102BD
:1000C0000976150026FF00952075089102C00501EC
:1000D0000980A101850319012AB700150126B7007F
:1000E000950175108100C0050C0901A10185041955
:1000F000012AA002150126A002950175108100C0F9
:100100000660FF0961A1010962150026FF00952024
:10011000750881020963150026FF00952075089176
:1001200002C005010906A101050719E029E715002C
:100130002501950875018102950175088101050762
:10014000190029FF150026FF009506750881000596
:10015000081901290595057501910295017503910D
:1001600001C00000000000000000000000000000CE
:10017000000000000000000000000000000000007F
:100180000000000000007E0F00D4FFFFFFC700004A
:10019000007800000000000000002A2B280000006A
:1001A0000000000000000000000000000029000026
:1001B00000002C1E3420212224342627252E362D03
:1001C0003738271E1F202122232425263333362E9D
:1001D00037381F0405060708090A0B0C0D0E0F100F
:1001E0001112131415161718191A1B1C1D2F313054
:1001F000232D350405060708090A0B0C0D0E0F10F8
:100200001112131415161718191A1B1C1D2F313033
:10021000354C726762206D617472697820746F6703
:10022000676C65205B25735D3A207267625F6D6164
:10023000747269785F636F6E6669672E656E61625E
:100240006C65203D2025750A0044454255473A20FB
:1002500064697361626C65642E0A004445425547C7
:100260003A20656E61626C65642E0A004F6E65739C
:10027000686F743A206163746976653A2025640A70
:10028000000A002530325820006B6579626F617278
:10029000645F7265706F72743A20005461726765B2
:1002A0007420636F6E6E65637465640D0A0054613B
:1002B0007267657420646973636F6E6E65637465DD
:1002C000642C207468726F74746C696E6720636F3D
:1002D0006E6E656374696F6E20617474656D7074A1
:1002E000730D0A004661696C656420746F2065783F
:1002F00065637574652025730A007267625F6D61BE
:10030000747269785F636F6E6669672E666C616789
:1003100073203D2025640A007267625F6D6174720C
:1003200069785F636F6E6669672E737065656420B8
:100330003D2025640A007267625F6D61747269789E
:100340005F636F6E6669672E6873762E76203D2038
:1003500025640A007267625F6D61747269785F6319
:100360006F6E6669672E6873762E73203D20256454
:100370000A007267625F6D61747269785F636F6EA5
:100380006669672E6873762E68203D2025640A0012
:100390007267625F6D61747269785F636F6E6669C0
:1003A000672E6D6F6465203D2025640A00726762C8
:1003B0005F6D61747269785F636F6E6669672E65E1
:1003C0006E61626C65203D2025640A007267625F81
:1003D0006D61747269785F636F6E66696720454509
:1003E00050524F4D0A007267625F6D617472697896
:1003F0005F696E69745F6472697665727320726793
:10040000625F6D61747269785F636F6E6669672E93
:100410006D6F6465203D20302E2057726974652011
:1004200064656661756C742076616C7565732074A3
:100430006F20454550524F4D2E0A007267625F6D26
:1004400061747269785F696E69745F6472697665F8
:100450007273206565636F6E666967206973206ECD
:100460006F7420656E61626C65642E0A005B735D5B
:10047000000A0025303862003A200025303258004A
:100480000A722F632030313233343536370A000A8E
:100490000025303258006B6579626F6172645F735A
:1004A00065745F6C65643A2000000101010101017F
:1004B000010101020202020202020202030303031B
:1004C00003030303040404040404040505050505EB
:1004D00006060606060707070707080808080909A9
:1004E00009090A0A0A0B0B0B0C0C0C0D0D0D0E0E54
:1004F0000E0F0F0F101011111112121313141415E7
:100500001516161717181819191A1A1B1B1C1D1D5A
:100510001E1E1F20202122222324242526262728B0
:1005200029292A2B2C2D2D2E2F30313232333435E0
:10053000363738393A3B3C3D3E3F404142434445E3
:10054000464748494A4C4D4E4F50515354555658C2
:10055000595A5B5D5E5F616264656668696B6C6D6C
:100560006F7072737577787A7B7D7E8082838587E2
:10057000888A8C8E8F91939596989A9C9EA0A2A320
:10058000A5A7A9ABADAFB1B3B5B7BABCBEC0C2C425
:10059000C6C9CBCDCFD1D4D6D8DBDDDFE2E4E7E9E5
:1005A000EBEEF0F3F5F8FAFDFF6565636F6E6669D3
:1005B000675F7570646174655F7267625F6D6174B7
:1005C0007269785F64656661756C740A0029001E43
:1005D000001F002000210022002B0014001A000838
:1005E0000015001700E00004001600070009000ACB
:1005F00000E1001D001B00060019000500000000BE
:1006000000E300105F28004A002A0027002600258A
:1006100000240023004C00130012000C0018001CE2
:1006200000340033000F000E000D000B00E5003811
:1006300000370036001000110000000000E6001135
:100640005F2C004D0035021E021F022002210222F3
:1006500002005C1E001F002000210022004C00014F
:100660000050004F0052002F00C05C01000100014B
:100670000051002F0200000000010001004C002684
:10068000022A002702260225022402230201002753
:1006900000260025002400230031022E025E005DAA
:1006A000005C00300001002D005B005A0059003052
:1006B0000200000000620001004C00270245003AE1
:1006C000003B003C003D003E00C25C1E021F0220B9
:1006D0000221022202C35CAC00AB00A9004B002D3A
:1006E00002A800AD00AE00AA004E002D00000000E0
:1006F00000010001000100260244004300420041C5
:100700000040003F000100270226022502240223A8
:10071000023100C95CC75CC55C4A002E000100CAFA
:100720005CC85CC65C4D002E0200000000010001A8
:1007300000010001000100010001000100010001B1
:1007400000010001000100010001000100010001A1
:100750000001000100010001000100010001000191
:100760000001000100000000000100010001000183
:100770000001000100010001000100010001000171
:100780000001000100010001000100010001000161
:100790000001000100010001000100010001000151
:1007A000000000000001000100010001005B435D4A
:1007B000005B445D005B535D005B575D005B525D19
:1007C0000009027B00040100A0FA090400000103F3
:1007D00001010009211101000122400007058103E8
:1007E00008000A09040100020300000009211101A8
:1007F00000012222000705820320000107050303F0
:100800002000010904020001030000000921110178
:1008100000012232000705840320000A09040300B6
:100820000203000000092111010001222200070536
:1008300085032000010705050320000112010002C5
:100840000000000810CB56620006010200011803E8
:1008500049007200690073002000520065007600B4
:100860002E002000360000000E034B0065006500DE
:10087000620069006F0000000403090472676220CF
:100880006D61747269782073657420737065656436
:10089000205B25735D3A2025750A00726762206D22
:1008A00061747269782073657420687376205B25A3
:1008B000735D3A2025752C25752C25750A00726705
:1008C00062206D6174726978206D6F6465205B25AC
:1008D000735D3A2025750A0011241FBECFEFDAE0C0
:1008E000DEBFCDBF04B603FE27C0809122059091E4
:1008F0002305A0912405B09125058730904BA74092
:10090000B04BD1F4109222051092230510922405C9
:100910001092250514BE84B7877F84BF0FB6F89464
:10092000A8958091600088618093600010926000BB
:100930000FBEE0E0F8E3099513E0A0E0B1E0E4EEDB
:10094000FBE602C005900D92A430B107D9F725E06F
:10095000A4E0B3E001C01D92A232B207E1F70E9409
:10096000952C0C9496350C940000FF93EF93E09136
:100970000403F0910503309709F00995EF91FF9179
:100980000895FC018591803011F0EFDFFBCF0895D1
:10099000FF27E0E230E247FF0CC0419597FF09C016
:1009A000EDE26095709580959095611D711D811D9A
:1009B000911D27FF02C0219530E350E2AA27660F60
:1009C000771F881F991FAA1FA41710F0A41B6395F7
:1009D0005A95A9F7AA3008F0A95FA05DAF93F395E7
:1009E000611571058105910541F7ED3211F4EF9321
:1009F000F395F21718F43F93F395FBCF8F91B5DF82
:100A0000FA95E1F70895E991F9918591803021F007
:100A1000853219F0AADFF9CF089520E0E8945591C6
:100A20005532C1F3503311F4689455915A3348F458
:100A3000505390F3220F022E220F220F200D250F6C
:100A4000F4CF0EF4219589919991533619F35337C8
:100A500029F1533559F1BC0188279927E8945C3670
:100A600021F48991999168945591543639F446EF5F
:100A70007EF077FF0DC08FEF9FEF0AC055374AE039
:100A800039F0583540E121F0523642E009F008953E
:100A9000FF93EF937DDFEF91FF91B7CFFF93EF933C
:100AA000FC0181918030B9F360DFFBCFFF93EF93BE
:100AB00068DFF1CFDF93CF93CDB7DEB72596A3DF05
:100AC000CF91DF910895E8EDF0E080818E7F808303
:100AD0001092E2001092DA001092E100A0EEB0E075
:100AE0008C9181608C9380818F77808319BCA7ED76
:100AF000B0E08C918E7F8C9380818F7E808310926A
:100B0000D20408952091E4003091E50095E6A90112
:100B10002091EC00822F817020FF06C08091E800B8
:100B200080FF06C080E008952091E80022FD1AC0F1
:100B30008091DF04882389F0853089F08091EB0073
:100B400085FD0FC02091E4003091E5004217530766
:100B5000F9F29150E1F684E0089582E0089583E08F
:100B6000089581E00895EF92FF920F931F93CF9322
:100B70007C018B010E948205C82F811117C08091D2
:100B8000E80085FD0BC08091E8008E778093E80037
:100B90000E948205882399F3C82F08C0F70181912C
:100BA0007F018093F1000150110949F78C2FCF91FB
:100BB0001F910F91FF90EF9008958091E10487FFBE
:100BC00013C08091E80082FF06C08091E8008B7717
:100BD0008093E80004C08091DF048111F2CF089572
:100BE0008091DF048823D9F38091E80080FFF8CF5B
:100BF0008091E8008E77ECCF982F9093E900242F16
:100C0000762F50E0891731F07091EC002091ED00C3
:100C10005091F00021FD07C09F5F973071F78093DE
:100C2000E90081E008953091EB003E7F3093EB00C6
:100C30003091ED003D7F3093ED003091EB0031605D
:100C40003093EB007093EC002093ED005093F00094
:100C50002091EE0027FDE0CF80E00895CF92DF9253
:100C6000EF92FF920F931F93CF93DF93C8EDD0E0E5
:100C700088818F7E8883E7EDF0E0808181608083CA
:100C800084E082BF81E08093D20488818E7F888354
:100C900002EE10E0F80110821092DA0081EEC82E08
:100CA000D12CF601108288818F77888388818068B3
:100CB000888388818F7D888319BC1092DF0410920D
:100CC000E0041092DE041092DD0490EEE92EF12C87
:100CD000F70180818B7F808388818160888342E0F7
:100CE00060E080E00E94FC05F60180818E7F8083B9
:100CF000F801808181608083808188608083F70132
:100D000080818E7F8083888180618883DF91CF910D
:100D10001F910F91FF90EF90DF90CF900895FC010D
:100D20008091E7049091E80486179707A0F0611579
:100D3000710529F49091E8009E779093E80090E087
:100D40006115710551F4911108C08091E80082FF8E
:100D500034C080E00895BC01F2CF8091DF04882385
:100D6000C1F18530C1F18091E80083FD30C08091F0
:100D7000E80082FDEACF8091E80080FFE1CF80911A
:100D8000F3002091F200382F6115710519F0283019
:100D9000310558F091E02830310509F090E02091BC
:100DA000E8002E772093E800CBCF81918093F1006B
:100DB000615071092F5F3F4FE7CF8091DF04882397
:100DC00041F0853041F08091E80083FFBECF81E0A3
:100DD000089582E0089583E008950895089580912C
:100DE000D40408959C014FB7F8948091C804909161
:100DF000C904A091CA04B091CB044FBF821B930BCE
:100E000008952FB7F8946091C8047091C904809137
:100E1000CA049091CB042FBF08952FB7F894809106
:100E2000C8049091C904A091CA04B091CB042FBF0B
:100E300008959C01FC0132969FEF80E04191461796
:100E400051F09F3F19F4411101C0982F8F5F8630F8
:100E5000A9F79F3F09F40895290F311D97FD3A9591
:100E6000F901628308952091C5043091C6042817C2
:100E7000390771F09093C6048093C504E091C304D0
:100E8000F091C404309721F00084F185E02D09949D
:100E900008952091C1043091C2042817390771F0D8
:100EA0009093C2048093C104E091C304F091C40400
:100EB000309721F00680F781E02D09940895FC0118
:100EC000680F791F8FEF91E32191822728E030E0AE
:100ED00087FF09C0880F892721503109C9F7E61714
:100EE000F70791F70895880FF7CFFA01811101C034
:100EF000FB01099480935C018091F20483708093DC
:100F00005B010E94931683E080935E010895EF9247
:100F1000FF920F939701201B31092F3F310519F0E4
:100F200010F02FEF30E02095382F320F08F43FEF0C
:100F3000832F0F91FF90EF900895EF92FF920F9300
:100F40009701201B31092F3F310519F010F02FEFC9
:100F500030E0322F3095482F430F08F44FEF842FA5
:100F6000620F0F91FF90EF900895EF92FF920F9311
:100F7000972F093438F4B701601B71096F3F710571
:100F800019F010F06FEF70E0485F5F4F413151058D
:100F900040F0A901485F5F4F4131510510F06FEFFC
:100FA00070E06095482F460F08F44FEF842F37FF0D
:100FB00002C02D5F3F4F3595279535952795609158
:100FC000F304620F792F0F91FF90EF900895EF9245
:100FD000FF920F931F930E0D1F2D111DF90137FF67
:100FE00003C0F195E195F10924E0EE0FFF1F2A956A
:100FF000E1F7EF3FF10519F014F0EFEFF0E09A019F
:1010000057FF03C031952195310994E0220F331F1A
:101010009A95E1F72E173F070CF4F901E00FF11F45
:10102000EF3FF10519F010F0EFEFF0E0E095282F19
:101030003E2F230F08F42FEF822F1F910F91FF9067
:10104000EF900895EF92FF920F93970195E0099F1B
:10105000200D311D11242F3F310519F010F02FEF15
:1010600030E02095382F320F08F43FEF832F0F9197
:10107000FF90EF90089522E8241B08F420E0620F0F
:1010800008954095282F429F412D1124842F0895C3
:101090000F931F9310E0F801EE0FFF1FE85CFD4F68
:1010A0009081905797FD9195000F111FF801E45022
:1010B000FE4F05AD0052110B2003F001219FF00DF2
:1010C000112408E310E0091B110997FD1395400353
:1010D0009001419F300D1124E20FF31F9F01220F59
:1010E000331F2E0F3F1F37FF02C021583F4F220FE3
:1010F000232F221F330B620F1F910F9108950F931F
:101100001F93522F10E0F801EE0FFF1FE450FE4F27
:10111000A5ADA052BB0B9D015203F001539FF00DF2
:101120001124000F111FD801A85CBD4F0C9100576E
:10113000110B40039001419F300D11242E0F3F1FD2
:1011400037FF02C0215C3F4F96E0359527959A9571
:10115000E1F7620F1F910F9108950F931F93522F84
:1011600010E0F801EE0FFF1FE450FE4FA5ADA052B6
:10117000BB0B9D015203F001539FF00D1124000F92
:10118000111FD801A85CBD4F0C910057110B4003F3
:101190009001419F300D11242E0F3F1F37FF02C0D9
:1011A00021583F4F220F232F221F330B620F1F9115
:1011B0000F910895EF920F93972F23E0029FB001B4
:1011C0001124759567956E0D792F0F91EF90089505
:1011D000322F50E0FA01EE0FFF1FE450FE4F95ADA5
:1011E000905297FD9195440F551FFA01E85CFD4F11
:1011F0002081231B330B290F311D97FD3A95620F78
:101200000895E42FF0E0EE0FFF1FE450FE4F65ADB0
:10121000621B0895E42FF0E0EE0FFF1FE85CFD4F26
:101220006081621B0895622F0895E42FF0E0EE0FB5
:10123000FF1FE85CFD4F408134EE439F412D112498
:10124000E82FF0E050E0445E5F4FDA01A21BB109E5
:101250009D01B7FF03C031952195310993E0220F1D
:10126000331F9A95E1F7AF01421B530B9A0157FDCB
:1012700020E0582F259F212D1124822F0895E42F3F
:10128000F0E0EE0FFF1FE85CFD4F408134EE439F1E
:10129000412D1124E72FF0E050E0445E5F4FDA016A
:1012A000A21BB1099D01B7FF03C0319521953109FA
:1012B00093E0220F331F9A95E1F7AF01421B530BC6
:1012C0009A0157FD20E0279F212D1124722F0895A8
:1012D0000C946E0BFF920F931F93CF93DF93182FF5
:1012E000062FF42ED0E0C0E02F2D402F612FCE012D
:1012F0000E9468092196C434D105B1F7DF91CF91DE
:101300001F910F91FF900895FC019B01009729F414
:1013100080E077FF2BC080E80895AC0197FF04C000
:1013200044275527481B590BB901640F751F37FD1A
:1013300010C0241B350BC901A5E0880F991FAA9581
:10134000E1F70E94CC3480E2861BF7FF0FC0819545
:101350000895CB0165E0880F991F6A95E1F7BA01FE
:10136000621B730B0E94CC3480E6EECF0895EF929F
:101370000F93CF93DF93D72FC82FC9010E19BA014E
:101380000E948409602F681B7D2F8C2FDF91CF91E5
:101390000F91EF9008950F93CF93DF93D72FC82F1E
:1013A000C901BA010E948409682F600F7D2F8C2F1C
:1013B000DF91CF910F910895EF920F931F93CF93E9
:1013C000DF93D62FC72F182FC9010E19010FBA01AD
:1013D0000E948409081B202F219F212D1124822F78
:1013E0006D2F7C2FDF91CF911F910F91EF9008957A
:1013F000EF920F931F93CF93DF93D62F172FC82F02
:10140000C9010E19070FBA010E948409702F781BB9
:10141000719F712D11246D2F8C2FDF91CF911F9112
:101420000F91EF9008950F931F93CF93DF93D62FD3
:10143000C72F182FC901212F201B022FBA010E948C
:101440008409982F990F990F891B800F282F219FAE
:10145000212D1124822F6D2F7C2FDF91CF911F9191
:101460000F9108950F931F93CF93DF93D62F172FCC
:10147000C82FC901272F201B022FBA010E948409FF
:10148000982F990F990F782F791B700F719F712DDD
:1014900011246D2F8C2FDF91CF911F910F91089503
:1014A000E82F86FDE0952E2F2F7086FD2F5FE695A5
:1014B000E695E695E670F0E0E052FE4F9181929F4E
:1014C000902D212D112492959F702295207F922B93
:1014D0002081920F87FD919580E8890F0895AC01D6
:1014E0008230910508F408959FEF413E8EE1580740
:1014F00040F49A0195E0369527959A95E1F798E0A2
:10150000920F61E0E62FE90FFF27FF1F9F0135953E
:101510002795822F229FF001239FF00DF00D1124BB
:101520004E175F0738F49FEF920F961758F78FEF1B
:10153000860F08952F3FE9F361E0620FF6CF0F9316
:10154000CF93DF93D72FC82F47FD419588E390E0D5
:10155000841B910947FD9395889FB001899F700D69
:10156000700D1124229FC001239F900D900D112416
:10157000860F971F0E946F0A982F990F890F682F67
:10158000600F7D2F8C2FDF91CF910F91089530E068
:1015900020E0869F212D969F200D311D1124C90129
:1015A0000895AF92BF92CF92DF92FF920F931F9355
:1015B000CF93DF93362F472FE82FF0E0E755FB4F0F
:1015C00071110FC0E4918E2F2E2F6E2F722FDF918D
:1015D000CF911F910F91FF90DF90CF90BF90AF9070
:1015E0000895C72FD0E02491F22E022F10E056E08C
:1015F000659FC0011124EFEFF0E0BF010E94B834F5
:10160000832F90E0880F991F35E5369FD001379FD3
:10161000B00D11248A1B9B0B982F990F980F6F0107
:10162000CC1ADD0AC09ED001C19EB00DD09EB00D77
:1016300011248B2F499FA0011124452F55276F019D
:10164000C41AD50AC09EA001C19E500DD09E500D57
:1016500011245F01A91AB108AC9E6001AD9ED00CA7
:10166000BC9ED00C1124CD2CDD24EC19FD09E09F8B
:10167000E001E19FD00DF09FD00D1124ED2F6230DD
:101680007105A1F050F46115710509F49ECF613028
:10169000710581F0EB2F852F98CF6430710569F0CB
:1016A00080F06630710509F490CFF4CFE22F2B2F34
:1016B0008D2F8BCFE22F252F88CFEB2F822F2D2F31
:1016C00084CF2B2F8F2DE52F80CF789408955598B8
:1016D0005D9889B185FB882780F90895FF920F9363
:1016E0001F93CF93DF93EC01F62E042F122F0E944D
:1016F000670B81110FC0C232D10564F0A297FE01C1
:10170000EE0FFF1FEC0FFD1FEB50FC4FF18200832B
:10171000128307C00E94670B882389F3C232D10568
:1017200074F3DF91CF911F910F91FF900895CF93A4
:10173000C82F0E94670B882329F081E0C23228F06D
:1017400080E003C081E0C434D8F7CF9108952F9290
:101750003F924F925F926F927F928F929F92AF9241
:10176000BF92CF92DF92EF92FF920F931F93CF938E
:10177000DF93CDB7DEB728970FB6F894DEBF0FBE64
:10178000CDBF282E7C836B8320915F018EE0289F44
:10179000802D11248D83825F8983853410F034E499
:1017A00039830E94670B882329F08981833210F0E6
:1017B00092E299830E94670B811105C0ED81E232AC
:1017C00010F4F2E2FD832091F8042A839D81892F91
:1017D00090E098878F83880F991FFC01E450FE4F9B
:1017E0006F01822D90E09C012F5F3F4F3E832D8340
:1017F00089819F819817D0F028960FB6F894DEBFA4
:101800000FBECDBFDF91CF911F910F91FF90EF9051
:10181000DF90CF90BF90AF909F908F907F906F9010
:101820005F904F903F902F900C94970BEF81F8852D
:10183000E054FD4F8081909160018923F9F0309050
:10184000F3044090F4048D819E8188509B4F3C01AD
:10185000522C10E0FA815F16D8F02091F504129F07
:10186000112D1124632D742D812F0E94D10A462F32
:10187000282F672F8F8198850E9468092F813885CE
:101880002F5F3F4F38872F8332E0C30ED11CB0CF7C
:10189000F30181913F01F601A4ACA81ABB0885AC05
:1018A000F3018781881A9908AA9C9001AB9C300D9E
:1018B000300D1124889CC001899C900D900D11243D
:1018C000820F931F0E946F0A082F6091F60421E097
:1018D000620F08F46FEFF301EE0FFF1FE85FF440B3
:1018E000858996890E94C70A7C019401A501632D10
:1018F000742D812FEB81FC810995362E472E539450
:10190000182FA8CFCF92DF92EF92FF920F931F93E1
:10191000CF93DF937C01C0915F018EE0C89FC02D03
:1019200011241EE01C0F153408F014E40E94670B0C
:10193000882319F0133208F012E20E94670B81111C
:1019400003C0C23208F4C2E22091F60431E0230F52
:1019500008F42FEF30E050E040E06FEF7FEF80E0E1
:1019600090E00E94E0346901D0E001E02C2FC11723
:1019700058F0812FDF91CF911F910F91FF90EF9041
:10198000DF90CF900C94970BFE01E054FD4F8081C7
:1019900090916001892309F14091F8044150042E8F
:1019A000000C550B47FF1BC0C6016091F604600F89
:1019B00008F46FEF0E94C70AAC016091F3047091C4
:1019C000F4048091F504F70109950E94D10A462F8D
:1019D000282F672FCE010E9468092196C7CFFA01F0
:1019E000E850FB4F818982130AC0FA01EE0FFF1FF6
:1019F000E850FB4F818D928D8C159D05B0F24150C2
:101A00005109D0CFAF92BF92CF92DF92EF92FF9267
:101A10000F931F93CF93DF936C01C0915F018EE012
:101A2000C89FC02D11241EE01C0F153408F014E4CB
:101A30000E94670B882319F0133208F012E20E940B
:101A4000670B811103C0C23208F4C2E26091F60450
:101A5000669566958091EE049091EF040E94C70A06
:101A6000F82E80E48F0D0E94500A90E8B92EB80E2F
:101A70008F2D0E94500A20E8A22EA80ED0E0C11798
:101A800068F0812FDF91CF911F910F91FF90EF9020
:101A9000DF90CF90BF90AF900C94970BFE01E05475
:101AA000FD4F8081909160018923A1F06091F30442
:101AB0007091F4048091F504EF2C0C2F2A2D4B2DFE
:101AC000F60109950E94D10A462F282F672FCE01D3
:101AD0000E9468092196D3CF6F927F928F929F9236
:101AE000AF92BF92CF92DF92EF92FF920F931F932C
:101AF000CF93DF935C01C0915F018EE0C89FC02D42
:101B000011241EE01C0F153408F014E40E94670B2A
:101B1000882319F0133208F012E20E94670B81113A
:101B200003C0C23208F4C2E26091F6046695809167
:101B3000EE049091EF040E94C70AF82ED0E0CE0187
:101B4000880F991F9C0124503E4F6901C11788F0EE
:101B5000812FDF91CF911F910F91FF90EF90DF9038
:101B6000CF90BF90AF909F908F907F906F900C948C
:101B7000970BFE01E054FD4F808190916001892315
:101B800079F1F60184AD282F2057330B490185AD3B
:101B9000E82FE052FF0B3F01889C9001899C300D9B
:101BA000300D1124EE9FC001EF9F900D900D112478
:101BB000820F931F0E946F0A082F6091F3047091A7
:101BC000F4048091F504EF2C9301A401F50109952B
:101BD0000E94D10A462F282F672FCE010E94680944
:101BE000F2E0CF0ED11C2196B1CFBF92CF92DF92FF
:101BF000EF92FF920F931F93CF93DF936C01C091ED
:101C00005F018EE0C89FC02D11241EE01C0F15340B
:101C100008F014E40E94670B882319F0133208F0CF
:101C200012E20E94670B811103C0C23208F4C2E2C3
:101C30006091F60466958091EE049091EF040E9405
:101C4000C70AB82ED0E0CE01880F991F9C012450FE
:101C50003E4F7901C11760F0812FDF91CF911F9125
:101C60000F91FF90EF90DF90CF90BF900C94970B67
:101C7000FE01E054FD4F8081909160018923C1F005
:101C8000F70125AD2052330B44AD4057550B609101
:101C9000F3047091F4048091F5040B2DF60109957D
:101CA0000E94D10A462F282F672FCE010E94680973
:101CB000F2E0EF0EF11C2196CDCFEF92FF920F9341
:101CC0001F93CF93DF937C01C0915F018EE0C89F8B
:101CD000C02D11241EE01C0F153408F014E40E94DE
:101CE000670B882319F0133208F012E20E94670B89
:101CF000811103C0C23208F4C2E26091F604669515
:101D0000669521E0620F08F46FEF8091EE049091E8
:101D1000EF040E94C70A082FD0E0C11748F0812FB6
:101D2000DF91CF911F910F91FF90EF900C94970B43
:101D3000FE01E054FD4F808190916001892391F074
:101D40006091F3047091F4048091F504202F4C2FDE
:101D5000F70109950E94D10A462F282F672FCE013F
:101D60000E9468092196D9CFAF92BF92CF92DF929D
:101D7000EF92FF920F931F93CF93DF93182F8091D1
:101D80005C01811323C09091F204937020915B0158
:101D900030E081E09217130609F480E081708093AF
:101DA00061018091F70490916001981739F0809358
:101DB000600140E060E080E00E946A09133288F42C
:101DC000E12FF0E0E856FA4C0C94FF3481E0E6CFC6
:101DD00080916101882389F140E060E080E00E9409
:101DE0006A0980E02AC0C0915F018EE0C89FC02DC3
:101DF00011240EE00C0F053408F004E40E94670B78
:101E0000882319F0033208F002E20E94670B811167
:101E100003C0C23208F4C2E26091F3047091F4048A
:101E20008091F5040E94D10AF62EE72ED82ED0E03C
:101E3000C01708F1802F0E94970B90915F019F5F60
:101E400090935F0181110CC082E080935E018091CC
:101E50006101811105C0111103C083E080935E010F
:101E6000DF91CF911F910F91FF90EF90DF90CF9076
:101E7000BF90AF900895FE01E054FD4F8081909196
:101E80006001892331F02D2D4F2D6E2DCE010E9442
:101E900068092196CDCFC0915F018EE0C89FC02D0B
:101EA00011240EE00C0F053408F004E40E94670BC7
:101EB000882319F0033208F002E20E94670B8111B7
:101EC00003C0C23208F4C2E2E090F404F090F504DA
:101ED000D091F3046D2F7E2D8F2D0E94D10AD62E26
:101EE000C72EB82E6091F6046D0F7E2D8F2D0E94A7
:101EF000D10AF62EE72EA82ED0E0C01708F09ACF10
:101F0000FE01E054FD4F908180916001892359F0DA
:101F10002A2D4F2D6E2D90FD03C02B2D4D2D6C2D98
:101F2000CE010E9468092196E8CFC0915F018EE042
:101F3000C89FC02D11240EE00C0F053408F004E4F6
:101F40000E94670B882319F0033208F002E20E9416
:101F5000670B811103C0C23208F4C2E2E090F404BE
:101F6000D090F5042091F60450E4F52E3F2D329FD9
:101F7000312D1124F32ED0E0C01708F05BCFFE0105
:101F8000E054FD4F8081909160018923B9F0FE01FA
:101F9000EE0FFF1FE450FE4F85AD82958F7060916C
:101FA000F3048F9D600D11247E2D8D2D0E94D10A8A
:101FB000462F282F672FCE010E9468092196DCCF7B
:101FC000C0915F018EE0C89FC02D11240EE00C0F60
:101FD000053408F004E40E94670B882319F00332EB
:101FE00008F002E20E94670B811103C0C23208F4BC
:101FF000C2E2E090F404D090F5042091F60430E4BD
:10200000F32E3F2D329F312D1124F32ED0E0C01737
:1020100008F010CFFE01E054FD4F808190916001E7
:102020008923D9F0FE01EE0FFF1FE450FE4F64AD8F
:10203000F69EB001112495E0759567959A95E1F7A4
:102040008091F304680F7E2D8D2D0E94D10A462FBA
:10205000282F672FCE010E9468092196D8CFC09102
:102060005F018EE0C89FC02D11240EE00C0F0534D7
:1020700008F004E40E94670B882319F0033208F08B
:1020800002E20E94670B811103C0C23208F4C2E26F
:10209000F090F304D091F404E090F5046091F6041C
:1020A0006695669566958091EE049091EF040E9486
:1020B000C70A0E94500A805887FD8195880F282FF3
:1020C0003E2D239F212D1124822F6F2D7D2F0E94C5
:1020D000D10AF62EE72ED82ED0E0C01708F0AACEEF
:1020E000FE01E054FD4F808190916001892331F021
:1020F0002D2D4F2D6E2DCE010E9468092196EDCF1A
:102100008FE399E00E945D0E98CE85E199E0FACFC9
:1021100082E39AE00E94F50D90CE83E19AE0FACF37
:1021200088EF99E00E946C0D88CE8CED99E0FACF93
:1021300083E199E0E7CF8AE099E0E4CF81E099E09C
:10214000E1CF88EE98E0DECF8AED98E0EBCF8FE923
:102150009AE0E0CF8BEC99E0DDCF87EB99E0E2CF1E
:102160008DEA98E00E94020D68CE8FE798E0FACFE2
:1021700088E498E0F7CF81E498E00E94820C5DCE7D
:102180008BE398E0FACF8091F80421E0382F321BDE
:1021900008F430E0832F62E278E00E94A70B4DCE76
:1021A00062E278E080E0F9CF8091F80421E0382FF6
:1021B000321B08F430E0832F67EE77E0EECF67EE56
:1021C00077E0F0CF8091F80421E0382F321B08F43B
:1021D00030E0832F65EB77E0E0CF65EB77E0E2CF8F
:1021E0008091F80421E0382F321B08F430E0832F6F
:1021F0006DE977E0D2CF6DE977E0D4CF8091F80434
:1022000021E0382F321B08F430E0832F67E877E0B5
:10221000C4CF67E877E0C6CFF894E82FE295EF7077
:10222000F0E031A1282F2F7081E090E001C0880FED
:102230002A95EAF7982F9095932391A392A1892B41
:1022400082A30C94650B90919E0392FF06C0282FE9
:1022500028712830F9F4877F846093FF06C0282F07
:1022600028712831F1F4877E846120919F0320FF3B
:1022700006C0382F38713830D9F4877F816021FF4C
:1022800006C0282F28712831D1F4877E816194FD02
:10229000877E0895282F24712430F9F68B7F88607B
:1022A000DCCF282F2471243101F78B7E8861DDCFAC
:1022B000382F3171313019F78E7F8860E0CF282FA9
:1022C0002171213121F78E7E8861E1CFCF93DF9399
:1022D000EC0182389105A9F1D8F58133910509F413
:1022E00096C048F58932910509F48AC08A9709F4A5
:1022F00095C0C11522E5D20708F0B6C0C11531E579
:10230000D30708F026C1C83ED10508F09CC0C03EE6
:10231000D10560F5C83AD10508F087C0C53AD105A6
:1023200008F0EFC0C130D10509F12097F9F0C430B1
:10233000D105E0F440C08533910509F45AC0C9972E
:10234000C1F680919E03837089F0C0EED0E00EC08C
:10235000833E910599F170F4803E910501F1823E32
:10236000910539F680919E0382FD21C0CE01DF9157
:10237000CF910895863E910561F1873E910571F1F7
:10238000843E910509F0B5CF80919F0381FFEECF88
:1023900080919E03C7EED0E084FD0DC0E7CF809111
:1023A0009E0380FD07C190919F0390FFDFCFC3EE96
:1023B000D0E084FFDBCFD0E0C0E0D8CF80919E0397
:1023C00082FDFBC090919F0390FDBFCF84FFCECFD5
:1023D000F2CF80919E0383FDDDCFC8CF80919E0315
:1023E00083FDEEC090919F0391FFF0CFC4EED0E04B
:1023F000BDCF80919E0385FFB9CFC9E2D0E0B6CFB3
:1024000080919E0385FFB2CFC5E3D0E0AFCF80912E
:102410009E0386FFABCFCAE2D0E0A8CF80919E0397
:1024200086FFA4CFC1E3D0E0A1CFCF3BD10518F602
:10243000C85AD0E0CC0FDD1FC056DE4F0990D881BE
:10244000C02DD46493CFC11540E5D40708F064C013
:10245000C11580E4D80708F05CC0CE019A958115BB
:102460009F4108F483CFA7CFC11536E5D30718F5F0
:10247000C11545E5D40708F084C0C11584E5D80727
:1024800008F07AC09C2F969596959E01237033276D
:10249000C115D34508F462C0C1E0D0E002C0CC0F42
:1024A000DD1F2A95E2F730E2939FC0011124C82B6B
:1024B000D92BDA685BCFC1158AE5D80778F4C11546
:1024C00099E5D90708F068C0C11528E5D20708F4D6
:1024D00072CFDC2FCC27C06FD06A48CFCE01905688
:1024E0008115904208F067CF8D2F8F710E942311C4
:1024F00090E0982F882788279F719C012C2BE90159
:1025000049C0C55AD0E0C356DE4FC881D0E0D06480
:102510002DCFDF70D06A2ACFCE01E4E09695879563
:10252000EA95E1F783702C2F26952695237040E2DB
:10253000249F90011124382B8C2F8370C1E0D0E0B0
:1025400002C0CC0FDD1F8A95E2F7C22BD32BDC68CB
:102550000DCFDC2FCC27C16FD06A08CFC1E0D0E00F
:1025600002C0CC0FDD1F2A95E2F720E2929FC00146
:102570001124C82BD92BEBCFDC2FCC27C46FD06A0A
:10258000F5CE8C2F0E942311C82FD0E0DC2FCC2752
:10259000CC27DF71D062EACE8C2F8F700E9423117E
:1025A00034E0D695C7953A95E1F7CF709C2FEC01B2
:1025B000D069DCCEC9E3D0E0D9CEC2EED0E0D6CE31
:1025C000C6EED0E0D3CE0C94010780916403811154
:1025D00010926403089580959091630398239093DB
:1025E0006303089580915F0390912E03981301C0B7
:1025F00008958F5F8770FACFE92FEE0FE90FEE0F86
:102600008E0F982F977086958695869523E0829FEA
:10261000F0011124E05FFC4F50E040E080E02191A8
:1026200030E0092E02C0369527950A94E2F7217012
:102630003327042E01C0220F0A94EAF7822B4F5F42
:102640005F4F4330510559F70895E92FEE0FE90F19
:10265000EE0F8E0F982F977041E001C0440F9A95AE
:10266000EAF786958695869593E0899FF001112477
:10267000E05FFC4F30E020E070E05191DF01119706
:10268000CB01022E02C0969587950A94E2F78170DD
:1026900081958527842385278C932F5F3F4F233097
:1026A000310559F70895829590E09C01220F331F60
:1026B000220F331F2C7C959587959595879583736D
:1026C000282B30E0C901880F991F8A7A3595279504
:1026D0002575822B08959091F204937031F1811148
:1026E00025C094609093F20410925E018091EC04F6
:1026F00081608093EC048091ED0480FF16C080918E
:10270000F204869586951F928F938BE691E09F93B6
:102710008F938EEB98E09F938F930E945A050F90B2
:102720000F900F900F900F900F900895833210F03C
:102730009868D8CF880F880F982BD4CF8091F20457
:1027400086958695815009F482E20C946B138091F2
:10275000F204869586958F5F833208F081E00C94B1
:102760006B132091F204237059F18093F30460936A
:10277000F404413A08F040EA4093F5042091EC0457
:1027800021602093EC042091ED0420FF19C01F92DA
:102790004F931F926F9399279F938F938BE691E0AE
:1027A0009F938F938BE998E09F938F930E945A0594
:1027B0008DB79EB70A960FB6F8949EBF0FBE8DBF19
:1027C0000895E2EFF4E0438120E1421B08F440E089
:1027D0008181628190E00C94B113E2EFF4E04381D7
:1027E00020E1420F08F44FEF8181628190E00C9468
:1027F000B113E2EFF4E0628120E1621B08F460E0D3
:102800008181438190E00C94B113E2EFF4E06281A6
:1028100020E1620F08F46FEF8181438190E00C9416
:10282000B113E2EFF4E08181438162818850990B1A
:102830000C94B113E2EFF4E0818190E04381628176
:1028400008960C94B1138093F6049091EC04916077
:102850009093EC049091ED0490FF12C01F928F931F
:102860008BE691E09F938F938CE798E09F938F93F3
:102870000E945A050F900F900F900F900F900F909D
:1028800008958091F60420E1382F321B08F430E0DF
:10289000832F0C9423148091F60420E1382F320FFB
:1028A00008F43FEF832F0C942314EF92FF920F93C1
:1028B0001F93CF93DF938091630390916203892BE1
:1028C00090916103892B809306039091640399236F
:1028D00091F0892B8093060320E088E093E0FC01CF
:1028E0003191CF0131112F5FF3E08E309F07B9F79F
:1028F00021110E94E512E091C304F091C4043097C5
:10290000C9F10280F381E02D86E093E00995809182
:10291000ED0482FF2FC080FF04C089E892E00E948E
:10292000C104C6E0D3E08EE0E82E83E0F82E03E891
:1029300012E08091ED0480FF0BC088811F928F937D
:102940001F930F930E945A050F900F900F900F90B6
:102950002196EC16FD0669F78091ED0480FF0AC010
:1029600081E892E0DF91CF911F910F91FF90EF905E
:102970000C94C104DF91CF911F910F91FF90EF90C4
:10298000089590E080E00E94490790E080E00E9476
:10299000330710926203109261030C9455148093D4
:1029A00021050C94C11480912105982F96709630C2
:1029B00019F488600C94CF14877FFCCF21E030E0BD
:1029C00001C0220F8A95EAF7209580912105822384
:1029D0000C94CF14909160038095892380936003B9
:1029E000282F277091F4282F082E000C330B9217F4
:1029F000130659F090919F0392FD07C08595859528
:102A000085950E94DE1410926003089521E030E065
:102A100001C0220F8A95EAF780912105822B0C9440
:102A2000CF14809365030C94C114882321F00E9475
:102A3000EB120C9455140895882339F09091630398
:102A4000982B909363030C9455140895882381F177
:102A50009CEF980F913A78F4E8E0F3E02EE033E051
:102A60009191891303C0DF0111971C922E173F0724
:102A7000B9F70C94551490E2980F983050F4877081
:102A800091E001C0990F8A95EAF7892F0E94EB1215
:102A9000F0CF9BE5980F933020F490E080E00C9409
:102AA0004907885A873120F490E080E00C9433077E
:102AB0000895CF93C82F882309F44EC08CEF8C0F54
:102AC000813AF8F4E8E0F3E08EE093E0DF012D9145
:102AD000C21759F08A179B07D1F76C2F86E093E055
:102AE0000E941907CF910C9455142191C21303C071
:102AF000DF0111971C928E179F07B9F70E9455149A
:102B0000ECCF80E28C0F883068F4C77021E030E0B1
:102B100001C0220FCA95EAF780916303822B80934C
:102B20006303E0CFEBE5EC0FE33040F4F0E0E35675
:102B3000FE4F808190E0CF910C944907C85AC7316D
:102B400058F4EC2FF0E0EE0FFF1FE056FE4F8081AF
:102B50009181CF910C943307CF9108959FB7F8944A
:102B60001092D0049FBF9091DF04943009F048C0C8
:102B70002091E9002F703091EC00932F917030FD7F
:102B800090E8922B25E02093E9002091EB0020FFB4
:102B900034C02091EE0027FF30C02091CF042223C3
:102BA00021F02091E80025FF28C01092CF0426E0F4
:102BB0003091E80035FF14C08093F1008091E80067
:102BC00085FD27C08091E80080FFFCCF8091E80060
:102BD0008E778093E8009F709093E90080E00895DD
:102BE0003091DF04343049F43091EB0035FD05C0FD
:102BF000215041F481E08093CF049F709093E900CD
:102C00008FEF0895EFE9FFE03197F1F700C0000082
:102C1000CFCF8FB7F89421E02093D0048FBFDBCFC4
:102C20008093CC047093CE046093CD048091DF0434
:102C30008430F9F48093E9008FEF9091E80081509F
:102C400095FD06C095ED9A95F1F700008111F5CF3D
:102C50008091E80085FF0DC050E040E063E070E047
:102C60008CEC94E00E94B3058091E8008E7780930D
:102C7000E8000895BC0184E00C941016BC0183E0C8
:102C80000C941016CF93DF93EC0181E08093E90060
:102C90008FEF9091E800815095FD06C095ED9A95D3
:102CA000F1F700008111F5CF8091E80085FF14C095
:102CB00050E040E068E070E0CE010E94B3058091F2
:102CC000E8008E778093E80088E0FE01A5EDB4E08F
:102CD00001900D928A95E1F7DF91CF91089581E0FF
:102CE0008093E00080E28093D8001092C9008FE1C9
:102CF0009EE40197F1F700C0000087E090EBDC0153
:102D00008093220590932305A0932405B093250575
:102D100088E19CE00FB6F894A895809360000FBE00
:102D200090936000FFCF6E9A3EB13F7B2EB120643E
:102D30004FB7F89485EF93E0FC015191CF0168E023
:102D40002EB9000000C057FF3EB9550F000000C06B
:102D500000C000C03EB900C06A9591F7F4E0813C24
:102D60009F0751F74FBF8FE594E00197F1F700C03F
:102D7000000008957F928F929F92AF92BF92CF9260
:102D8000DF92EF92FF920F931F93CF93DF937C011B
:102D90005B01842E752E69018091710301E010E0C2
:102DA0008A3010F40AE010E0C1E0D0E0F894B501F8
:102DB000C701F6010995982E0E94650B911014C069
:102DC00021960C171D07FCF48091ED0480FF0CC0C8
:102DD0007F928F9284EE92E09F938F930E945A0588
:102DE0000F900F900F900F90892DDF91CF911F9131
:102DF0000F91FF90EF90DF90CF90BF90AF909F909A
:102E00008F907F900895CC9F9001CD9F300D300D15
:102E1000112490E080E045E34A95F1F70000019627
:102E200028173907C1F7C2CF80917003811110C0F4
:102E30008091D80080618093D8008AE18A95F1F76B
:102E400000C08091D90080FF0AC081E080937003A8
:102E500081E090917003913009F080E0089582E064
:102E6000809370030E9463051092DF04F1CF0E94EB
:102E70001417882351F0E091C304F091C4043097F3
:102E800021F00190F081E02D099480E008950F93E6
:102E90001F930E941417882321F01F910F910C9407
:102EA00001070E94010700919A0310919B03209152
:102EB0009C0330919D03600F711F821F931F1F9110
:102EC0000F910895CF92DF92EF92FF926B017C01F8
:102ED0000E9414178823A1F02FB7F8946091C804BA
:102EE0007091C9048091CA049091CB042FBF6C19D2
:102EF0007D098E099F09FF90EF90DF90CF90089594
:102F00000E944717F4CF1F93CF93DF93182FD0E081
:102F1000C0E0893311F4C0E5D0E0812F0E9459153B
:102F2000209731F4812FDF91CF911F910C942615BA
:102F30008FE99FE00197F1F700C000002197F0CFE3
:102F40000F931F93CF93DF93C62FD42F022FFC0133
:102F500082818823A1F06093EB040E940D07909377
:102F6000EA048093E904C77081E001C0880FCA9524
:102F7000EAF7DF91CF911F910F910C941C1580916E
:102F8000EB04681335C08091E9049091EA040E9433
:102F9000F206883C910560F510E21D0FCD17B9F0DF
:102FA00080E28C0F883040F4C77081E001C0880F48
:102FB000CA95EAF70E941515183048F481E09D2F54
:102FC000977001C0880F9A95EAF70E941C15802F10
:102FD0000E948317183098F4D77081E001C0880FE1
:102FE000DA95EAF7DF91CF911F910F910C941515A7
:102FF000C77081E001C0880FCA95EAF7F3CFDF916F
:10300000CF911F910F910895811108C089EA611134
:1030100001C08AEA0E94831780E008958130E1F7B9
:103020008EE46111F7CF8BE4F5CFCF93DF93C7E048
:10303000D2E060E0CE010E945C352196C11584E0AB
:10304000D807B9F7DF91CF9108956F927F928F9251
:103050009F92AF92BF92CF92DF92EF92FF920F9327
:103060001F93CF93DF938DECC82E85E0D82E9BEA7B
:10307000E92EF12CE701C857D10936011BC0F50133
:1030800085909490692DC8010E945C35682DC80117
:1030900001960E945C3582E0A80EB11C0E5F1F4FA6
:1030A000C017D10761F78CE0680E711C2C96CE1505
:1030B000DF0529F08E010C5011095301E0CF7E018C
:1030C00088E7E80EF11C88E7C80ED11C8BE8E816EB
:1030D00082E0F80679F6DF91CF911F910F91FF9072
:1030E000EF90DF90CF90BF90AF909F908F907F90A8
:1030F0006F900895CF93C82F6FEF811162E283E242
:1031000090E00E945C356FEFC11162E084E290E0D4
:103110000E945C356FEFC11169E185E290E0CF91CB
:103120000C945C3580E00E947A1860E086E290E0C2
:103130000E945C350E9425180E94151881E00C94AD
:103140007A18CF93DF93D82FC0919F03C2FB8827B3
:1031500080F98D1711F1D0FBC2F9C0939F036091E4
:103160009E0384E090E00E945C356C2F82E290E048
:103170000E945C3582E00E94EA148091ED0480FF99
:103180000CC01F92DF938CE692E09F938F930E9476
:103190005A050F900F900F900F90DF91CF910895E7
:1031A0000F931F93CF93DF93C42FD0E0CC0FDD1F7D
:1031B0002CE0629FC00DD11D112438E7839FC00D04
:1031C000D11D1124CE0187960E943E35082F10E0B4
:1031D000102F0027CE0188960E943E359801282B9B
:1031E000C901DF91CF911F910F910895462F84302F
:1031F00038F47A3028F4663018F4672F0C94D0181D
:1032000090E080E00895CF92DF92FF920F931F939A
:10321000CF93DF936C010091210580916503082B0A
:10322000C7E0D0E010E0FC2EC8010C2E02C095953E
:1032300087950A94E2F780FD0CC02197A0F7F12C46
:103240008F2DDF91CF911F910F91FF90DF90CF9045
:103250000895B6018C2F0E94F6180E9466110197FE
:1032600061F3EECFCF93DF93EC010E940319BE010F
:103270000E94F618DF91CF910C946611FC018081B9
:1032800091810E943219292F2F7092959F70925030
:103290009E3078F4E92FF0E0E554FA4C0C94FF34BA
:1032A000803F19F020F4883E20F481E00895843FA7
:1032B000E1F380E00895883EC0F3813FD1F7F5CF78
:1032C000822F869586958695089583E290E00E94E8
:1032D0003E35823289F484E290E00E943E358230AD
:1032E00059F485E290E00E943E3591E0893109F081
:1032F00090E0892F8170089580E0FCCFCF9384E027
:1033000090E00E943E35C82F82E290E00E943E3558
:10331000982F8C2FCF9108954F925F926F927F924A
:103320008F929F92AF92BF92CF92DF92EF92FF92D5
:103330006091F0037091F1038091F2039091F30397
:103340000E9462176B017C010E9447174B015C01D0
:103350008092F0039092F103A092F203B092F303F3
:10336000A091C703E7ECF3E08A2F90E04FEF5FEF07
:1033700060E070E04C195D096E097F09A91328C04F
:103380008093C7038091F403811135C09091F204BA
:10339000892F837019F0892F8695869590915E010B
:1033A000913009F441C0992341F1923009F44AC0A7
:1033B000933009F455C0FF90EF90DF90CF90BF900D
:1033C000AF909F908F907F906F905F904F900895F7
:1033D000218D328D2901712C612C4415550566050E
:1033E000770520F481509F5F3296C8CF2C0D3D1D8C
:1033F000328F218FF8CF80E0D1CF10925F01809281
:10340000EE049092EF04A092F004B092F10489E2ED
:10341000E7ECF3E0A8EFB4E001900D928A95E1F7B4
:1034200081E080935E01C7CFFF90EF90DF90CF9057
:10343000BF90AF909F908F907F906F905F904F90D4
:103440000C94B40EFF90EF90DF90CF90BF90AF90B0
:103450009F908F907F906F905F904F900C947A0721
:103460008091EC04882351F046E050E06CE170E07C
:1034700082EF94E00E944C351092EC046091EE04CF
:103480007091EF048091F0049091F1040E94621712
:10349000603171058105910508F48DCF10925E01B0
:1034A0008ACF8091ED0480FF08C089EA95E09F9360
:1034B0008F930E945A050F900F9085E38093F2043A
:1034C0008091620190916301A09164018093F30463
:1034D0009093F404A093F5048FE78093F6048FEFA4
:1034E0008093F70446E050E06CE170E082EF94E0F6
:1034F0000E944C351092EC04089510926303E8E0AA
:10350000F3E086E0DF011D928A95E9F70C94C1147F
:103510001F93CF93DF93CDB7DEB7AA970FB6F8947A
:10352000DEBF0FBECDBF81EE94E02091F100DC0143
:103530002D93CD01B4E0893E9B07B9F78091E20459
:10354000833009F472C0B8F4813009F449C0823084
:1035500009F4B3C08091E80083FF91C28091E10437
:103560009091E2049A3008F08AC2E92FF0E0E75324
:10357000FA4C0C94FF348A3009F48EC08B3009F475
:1035800071C0893039F78091E104813219F7809157
:10359000E5049091E604009711F00297D9F6809126
:1035A000E800877F8093E8008091E80082FF38C0C0
:1035B0009091F3008091F200029731F48091F10034
:1035C000813011F0863021F48091F1008093D40491
:1035D0008091E8008B778093E8000E94DD05BACFE8
:1035E0008091E104813A09F0B5CF8091E800877FAE
:1035F0008093E8008091E5049091E604892B61F4C2
:1036000068E085ED94E070E00E948F068091E8000C
:103610008B778093E8009ECF60E090E080E0F3CF6E
:103620008091DF048111C0CF95CF8091E104813A70
:1036300009F090CF8091E5049091E604892B09F080
:1036400089CF8091E800877F8093E8008091E8002F
:1036500080FFFCCF80915D018093F1008091E800B4
:103660008E77B9CF8091E104813209F073CF8091D8
:10367000E5049091E604892B09F06CCF8091E80075
:10368000877F8093E8000E94DD058091E3048093AA
:103690005D010E947D1A5ECF8091E104813209F0C4
:1036A00059CF8091E800877F8093E8000E94DD0574
:1036B0008091E4048093D3044DCF8091E104813A5A
:1036C00009F048CF8091E800877F8093E8008091DF
:1036D000E80080FFFCCF8091D304BECF803899F002
:1036E000823809F0CCC18091E5048F70873008F0F2
:1036F000C6C18093E9008091EB0085FB882780F9A3
:103700001092E90006C08091DD049091DE049111D1
:1037100082609091E800977F9093E8008093F10099
:103720001092F1008091E8008E77A5C1882309F4FA
:1037300093C1823009F0A3C18091E304811196C145
:103740008091E5048F702FEF280F263008F097C185
:103750008093E9002091EB0020FF88C1933031F481
:103760008091EB0080628093EB0080C19091EB0030
:1037700090619093EB0021E030E001C0220F8A9528
:10378000EAF72093EA001092EA008091EB0088604B
:10379000EACF811174C11091E3041F778091E30097
:1037A0008078812B8093E3008091E800877F80936D
:1037B000E8000E94DD058091E80080FFFCCF809149
:1037C000E30080688093E30082E0111183E080933E
:1037D000DF0455C18058823008F051C12091E304C4
:1037E0003091E4042C3DE3E03E07A1F583E08A83B9
:1037F0008AE289834FB7F894DE01139620E03EE019
:1038000051E2E32FF0E050935700E49120FF03C012
:10381000E295EF703F5FEF708E2F90E0EA30C0F0DE
:10382000C7968D939D932F5F243159F74FBF809199
:10383000E800877F8093E8006AE270E0CE0101969D
:103840000E948F068091E8008B778093E80017C173
:10385000C096E7CF8091E5049091E604432F552769
:103860004330510509F44AC078F54130510509F457
:103870007AC08BE790E0E1ECF7E04230510509F0C7
:10388000FEC02091E800277F2093E8002091E70404
:103890003091E8048217930708F49C0140E0211559
:1038A000310509F065C0411163C08091E80082FDD7
:1038B000C9CF8091DF04882329F2853019F28091E5
:1038C000E80083FFF2CFBECF4132510509F43CC07E
:1038D0004232510509F0D3C08430910508F0CFC0C1
:1038E000FC01EE0FFF1FE451FE4F0190F081E02D2F
:1038F00088519E4FDC018C9190E01AC03327213013
:103900003105D1F02115310561F02230310509F082
:10391000B6C0EEE4F8E0E4918E2F90E0EEE4F8E03B
:1039200007C0E8E7F8E0E4918E2F90E0E8E7F8E0E0
:10393000009709F4A4C0A5CFE8E6F8E0E4918E2F43
:1039400090E0E8E6F8E0F4CF8430910508F097C005
:10395000880F991FFC01EC50FE4F0190F081E02D83
:1039600089E090E08ECF82E190E0ECE3F8E089CF4F
:103970008091DF04882309F465CF853009F462CF94
:103980008091E80083FD5ECF8091E80082FD8DCFBD
:103990008091E80080FF83CF9091F3008091F20046
:1039A0002115310519F08830910550F041E0089754
:1039B00009F040E08091E8008E778093E8006FCFB7
:1039C00044914093F1003196215031090196E8CF9E
:1039D000803809F054C08091E800877F8093E80028
:1039E0008091E0048093F1009DCE811148C0109138
:1039F000E304123008F043C08091E800877F809391
:103A0000E8001093E0040E94DD05112311F084E02A
:103A100005C08091E30087FDFACF81E08093DF0449
:103A200042E061EC81E00E94FC0542E261EC84E04E
:103A30000E94FC0542E261EC82E00E94FC0542E249
:103A400060EC83E00E94FC0542E261EC85E00E94AC
:103A5000FC058091DF0413C08091E304813079F488
:103A600081E0933009F080E08093DE041092E90059
:103A70008091E800877F8093E8000E94DD058091B7
:103A8000E80083FF0AC08091E800877F8093E80008
:103A90008091EB0080628093EB00AA960FB6F894B9
:103AA000DEBF0FBECDBFDF91CF911F9108957F92F2
:103AB0008F929F92AF92BF92CF92DF92EF92FF923E
:103AC0000F931F93CF93DF93CDB7DEB72F970FB62A
:103AD000F894DEBF0FBECDBF8E010F5F1F4F8AE08F
:103AE000D8011D928A95E9F782E4C82E81E0D82E8C
:103AF000F12CE12CAA24A394B12C22E4822E21E003
:103B0000922EF60181916F018F3F09F443C0F89422
:103B1000E82FE295EF70F0E021A18F70A50102C0BF
:103B2000440F551F8A95E2F7CA01922F982B91A353
:103B300092A18095892382A30E94650B00C0ECE3CB
:103B4000F1E0712C31E021912F3F09F47AC0A22FCE
:103B5000A295AF70B0E090968C9190E02F7002C06B
:103B6000959587952A95E2F780FD6BC0832F782A7B
:103B7000330F8E169F0639F7F601319780818F3FFC
:103B800011F00E940C1150EA5A95F1F7F801EE0D70
:103B9000FF1D70828FEFE81AF80A95E0E916F1042C
:103BA00009F0AFCF4AE050E0B80180EA93E00E940C
:103BB00080357C01892B41F08AE0F801A0EAB3E06E
:103BC00001900D928A95E1F71091AB03E114F10495
:103BD000D1F181E0809368030E940D079093670301
:103BE0008093660380916603909167030E94F206BA
:103BF000059778F0A0EAB3E0E12FF0E0E354FC4F42
:103C000085EA93E02D9121938A179B07D9F71092AB
:103C1000680381E090E0EF28D1F02F960FB6F8947A
:103C2000DEBF0FBECDBFDF91CF911F910F91FF90EF
:103C3000EF90DF90CF90BF90AF909F908F907F904C
:103C4000089580E094CF809168038111CBCF0E94CA
:103C50001417D82EE091AB03DE011B967D0188235B
:103C600009F495C085E01D928A95E9F70E2F10E0C2
:103C700003541C4FC0907103B9E0BC1508F443C055
:103C800029E031E242E751E0B701C8010E94BA16CB
:103C9000882309F45BC023EB30E24FE751E0B70122
:103CA000C8010E94BA16882309F450C02BEA3FE1EC
:103CB00047E851E0B701C8010E94BA16882309F409
:103CC00045C02EE33FE142E951E0B701C8010E943F
:103CD000BA168823D9F1F9E0FC1508F44FC0109208
:103CE00071038091AA0390E045E050E0B70183544E
:103CF0009C4F0E94803521E020936F03892BC9F4EB
:103D0000D12C8D2D8ACF8091690390916A030E94F6
:103D1000F206843F914008F0B3CF80916F0388236F
:103D200009F4AAC085E0D7011D928A95E9F710929F
:103D30006F03A091AA03B0E0A354BC4F85E0FE013D
:103D40003B9601900D928A95E1F7DBCF809171034C
:103D50008F3F29F08F5F809371038A3010F20E94A9
:103D60000D0790936A03809369038091ED0480FFAF
:103D7000D4CF8EEA92E00E94C104CFCF8091ED04AF
:103D800080FFADCF8BE992E00E94C104A8CFF0E0A4
:103D9000E354FC4FF89485E0A4E8B3E001900D9261
:103DA0008A95E1F765E070E084E893E00E945F07A0
:103DB000809383030E94650BF894E091B003F0E0D8
:103DC000E355FC4F80818B8780938A0361E070E02C
:103DD000C7010E945F07809389030E94650BF894D6
:103DE000C0908B03D0908C03E0908D03F0908E03F5
:103DF00080916B0390916C03A0916D03B0916E0361
:103E0000C816D906EA06FB06D1F0C0926B03D09221
:103E10006C03E0926D03F0926E030E9414178111FF
:103E20000EC00E940107C61AD70AE80AF90AC09212
:103E30009A03D0929B03E0929C03F0929D030E9410
:103E4000650BF89486E0EFE8F3E0A2EFB4E00190B0
:103E50000D928A95E1F710919503112349F0809115
:103E6000F403811105C00E94B40E80E00E947A071D
:103E70001093F4030E94650B80E0CFCE0F931F9345
